:100000000C9441000C945E000C945E000C945E0015
:100010000C946B000C945E000C945E000C945E00DB
:100020000C945E000C9460000C945E000C9496029C
:100030000C945E000C945E000C945E000C945E00C8
:100040000C945E000C945E000C945E000C945E00B8
:100050000C945E00240108010C0126012A014401D0
:10006000480162016601800184019E01A201BC0178
:10007000C001DA01DE01F801FC01150219023202A9
:10008000380211241FBECFE5D4E0DEBFCDBF10E0A3
:10009000A0E6B0E0E8EAF6E002C005900D92AC38C8
:1000A000B107D9F710E0ACE8B0E001C01D92AB3C5D
:1000B000B107E1F70E9464020C9452030C94000013
:1000C0001F920F920FB60F921124C49A0F900FBE79
:1000D0000F901F9018951F920F920FB60F92112438
:1000E0008F9312BA88E085BB15BA12BA81E085BB3E
:1000F00015BAD9988F910F900FBE0F901F90189539
:10010000660F660F62BB282F30E0F901EE0FFF1F6C
:10011000EE0FFF1FE05AFF4F8381882359F4F90146
:10012000EE0FFF1FEE0FFF1FEE59FF4F808185BBC3
:1001300015BA0CC0813051F4F901EE0FFF1FEE0F1C
:10014000FF1FEE59FF4F808188BB18BAF901EE0FEF
:10015000FF1FEE0FFF1FE05AFF4F808180938C003E
:10016000818180938D0080918C00880F880F82BBE5
:1001700088E085BB15BA80918D00880F880F82BBFF
:1001800081E085BB15BA089590918C00E82FF0E0CE
:10019000EE0FFF1FEE0FFF1FE05AFF4F808180958B
:1001A000892380938C0090918D0081818095892393
:1001B00080938D0080918C00880F880F82BB88E02F
:1001C00085BB15BA80918D00880F880F82BB81E0B6
:1001D00085BB15BA0895682F893919F410928F00DC
:1001E00007C087FF05C0893919F08FEF80938F0012
:1001F00080918F00E82FF0E0E731F10508F063C14E
:10020000E65DFF4FEE0FFF1F0590F491E02D09947E
:100210006093950082E029C160938E0083E0809313
:100220008F00662389F09091950080919300981734
:1002300058F0209195008091930030E090E00A966C
:10024000821793070CF02BC181E00FC160939500DA
:1002500084E00BC160938E0085E080938F0066235D
:1002600089F09091950080919300981758F0209113
:1002700095008091930030E090E00A9682179307F2
:100280000CF00DC183E0F1C06093950086E0EDC0F5
:1002900060938E0087E080938F00662389F09091B1
:1002A000950080919300981758F0209195008091C7
:1002B000930030E090E00A96821793070CF0EFC0AD
:1002C00085E0D3C06093950088E0CFC060938E0036
:1002D00089E080938F00662389F09091950080914A
:1002E0009300981758F0209195008091930030E08A
:1002F00090E00A96821793070CF0D1C087E0B5C052
:10030000609395008AE0B1C060938E008BE080938B
:100310008F00662389F09091950080919300981743
:1003200058F0209195008091930030E090E00A967B
:10033000821793070CF0B3C089E097C060939500D3
:100340008CE093C060938E008DE080938F006623D5
:1003500089F09091950080919300981758F0209122
:1003600095008091930030E090E00A968217930701
:100370000CF095C08BE079C0609395008EE075C05D
:1003800060938E008FE080938F00662389F09091B8
:10039000950080919300981758F0209195008091D6
:1003A000930030E090E00A96821793070CF077C034
:1003B0008DE05BC06093950080E157C060938E0034
:1003C00081E180938F00662389F090919500809160
:1003D0009300981758F0209195008091930030E099
:1003E00090E00A96821793070CF059C08FE03DC049
:1003F0006093950082E139C060938E0083E1809321
:100400008F00662381F0909195008091930098175A
:1004100050F0209195008091930030E090E00A9692
:1004200082179307E4F581E120C06093950084E191
:100430001CC060938E0085E180938F00662381F05D
:100440009091950080919300981750F0209195001D
:100450008091930030E090E00A9682179307FCF4B5
:1004600083E103C06093950086E180938F00089537
:1004700060938E008FEF80938F00662309F1909137
:100480009500809193009817D8F020919500809165
:10049000930030E090E00A96821793078CF0C4989E
:1004A000D99A80919500909193006695891B0E943E
:1004B00080008091910082BF8091920084BD089558
:1004C00085E180938F00089583E08ABB8FEF87BB1F
:1004D00084BB8EEF81BB89E08093900080E28093A3
:1004E000910080EF8093920080E3809393001092BC
:1004F000940083B7856083BF12BE89B7816089BFCE
:1005000085B5876085BD14BC89B7806489BF0E94AA
:1005100021037894C49AD89A15BA12BA89E085BB97
:1005200015BA0E94CF020E94EB00FBCF1F920F92E0
:100530000FB60F9211242F935F936F937F938F9336
:100540009F93AF93BF93EF93FF938CB180939800E9
:10055000809196008233A0F48091970020919600BC
:1005600090E0820F911D62E370E00E942B03FC017A
:1005700080919800E756FF4F80832F5F209396006D
:10058000FF91EF91BF91AF919F918F917F916F916B
:100590005F912F910F900FBE0F901F901895809133
:1005A00096008823E1F3F89480919600815080931F
:1005B000960080919700E82FF0E0E756FF4FE0812A
:1005C0008F5F8093970080919700823310F0109294
:1005D000970078948E2F0895FF920F931F93CF93D7
:1005E000DF93F82E192F062F0E94CF02482F2F2DB0
:1005F000312FC901EC0110E00150104004C04993B3
:100600000E94CF02482F9E012F19822F4A3021F0DD
:1006100090E0801791079CF31882DF91CF911F9192
:100620000F91FF9008955D9BFECF8CB90895FC015A
:1006300004C05D9BFECF8CB9319680818823C9F7B9
:100640000895539A549A579A80B5866880BD10BC15
:100650008FE189B9089597FB092E07260AD077FD07
:1006600004D00CD006D000201AF4709561957F4F0D
:100670000895F6F7909581959F4F0895AA1BBB1B8F
:1006800051E107C0AA1FBB1FA617B70710F0A61B92
:10069000B70B881F991F5A95A9F780959095BC01B3
:0806A000CD010895F894FFCF8D
:1006A800000180000010010101001000200002007C
:1006B80000040400000820000002040108004000B3
:0C06C800100008010200080104000201FB
:00000001FF
